:100000000C942A001895000018950000189500001F
:10001000189500001895000018950000189500002C
:100020001895000018950000189500000C944106E2
:10003000189500000C947D110C94AF1118950000D8
:1000400018950000189500001895000018950000FC
:10005000189500008FE58DBFCCEFECE44E2E88E0C4
:100060008EBFD7E0F7E05F2EEEEFF7E0A0E6B0E05E
:10007000A89584B7082E877F84BF88E1992781BD22
:1000800091BD88278D933197E9F788E089B980E0A1
:1000900080BD88E18AB9662484B7877F84BF88E100
:1000A00081BD80E081BD80E08ABB8CE187BB83EEAF
:1000B00088BB80E084BB8FEF85BB80EF81BB8FE086
:1000C00082BB87E886B980E087B9379A85E083BF2D
:1000D00081EB8FBD81E08EBD8FEF8ABD579A0E9464
:1000E000A612A5EAB1E0E6E5F5E20E94BD0FA7EA97
:1000F000B1E0E8E5F5E20E94BD0FA9EAB1E0EAE56A
:10010000F5E20E94BD0FADEAB1E0EEE5F5E20E9436
:10011000BD0FA1EBB1E0E2E6F5E20E94BD0FA5EB59
:10012000B1E0E6E6F5E20E94BD0FA9EBB1E0EAE638
:10013000F5E20E94BD0FADEBB1E0EEE6F5E20E9404
:10014000BD0FA1ECB1E0E2E7F5E20E94BD0FA5EC26
:10015000B1E0E6E7F5E20E94BD0FA9ECB1E0EAE705
:10016000F5E20E94BD0FADECB1E0EEE7F5E20E94D2
:10017000BD0FA1EDB1E0E2E8F5E20E94BD0FA5EDF3
:10018000B1E0E6E8F5E20E94BD0F81E080939901BD
:100190000895A4E1B1E08C91082F033211F00C9482
:1001A000D900A4E1B1E00E94D80E0E94E50E0C94A3
:1001B0006601A4E1B1E08C91082F0B3111F00C9491
:1001C000E900A4E1B1E00E94D80E0E94E50E0C9473
:1001D0006601A4E1B1E0E6E5F5E22FEF91E00E94CF
:1001E000D10FA3EAB1E00C930091A301003018F005
:1001F00011F00C94FD000C945201A4E1B1E0EAE886
:10020000F5E22FEF91E00E94D10F002F003080E047
:1002100010F009F081E08F934091A301A4E1B1E0D7
:10022000EAE8F5E22FEF91E00E94D10F002F0417CA
:1002300081E008F080E09F918923882311F40C94D9
:100240002D01A4E1B1E00E94D80E0E94E50E0E94AB
:1002500067010C9466010C945001E4E1F1E0009117
:10026000A301A4E5B1E00E948412A4E5B1E00E94DC
:100270004C12ABE9B1E00C9300919B01003011F0FE
:100280000C9448010E9467010C9466010C94500183
:10029000A4E1B1E00E94D80E0E94E50E0C94660124
:1002A0000C94660100919B01003011F00C945E01EA
:1002B0000E9467010C9466010C946601A4E1B1E010
:1002C0000E94D80E0E94E50E0C946601089581E00C
:1002D0008093DA01A4E5B1E088278C93A4E9B1E02A
:1002E00088278C93AEE9B1E0E2E5F5E20E9469115E
:1002F00080E090E0ACE9B1E08D939C93A4E1B1E0A3
:100300000E948C12082F0F93A4E1B1E0E5EAF1E01E
:10031000222791E00E94D10F402F0F91041BA3EAE6
:10032000B1E00C93A4E1B1E00E948C12EA2FFB2F04
:100330000091A3013197E01BF0400FEFA4E5B1E07D
:100340000E94841281E08093D9010091D901043088
:1003500018F011F00C94200281E4482FA9EDB1E0CF
:10036000AD90BB24A3E5B1E0AA0DBB1D0C91041711
:1003700081E008F480E08F938AE5482FA9EDB1E091
:10038000AD90BB24A3E5B1E0AA0DBB1D0C910417F1
:1003900081E010F009F080E09F9189238F9381E63E
:1003A000482FA9EDB1E0AD90BB24A3E5B1E0AA0DC3
:1003B000BB1D0C91041781E008F480E09F91892B0C
:1003C0008F938AE7482FA9EDB1E0AD90BB24A3E558
:1003D000B1E0AA0DBB1D0C91041781E010F009F0EB
:1003E00080E09F918923882311F40C941802A9EDD1
:1003F000B1E0AD90BB24A3E5B1E0AA0DBB1D8C918B
:10040000AAEDB1E0AD90BB24A3E9B1E0AA0DBB1DFC
:100410008C93AAEDB1E08C918F5F8C9380E0AAED74
:10042000B1E0AD90BB24A3E9B1E0AA0DBB1D8C9354
:10043000A9EDB1E08C918F5F8C9310F40C94A50121
:10044000A4E9B1E00E948C12082F033011F00C9443
:100450005E02E4E9F1E0A4E9B1E00E94711180E0FC
:100460008093D9010091D901093118F011F00C9451
:100470005E02E9EDF1E00191112744E050E00E94B5
:10048000900FE5EAF1E0E00FF11FA4E9B1E00E946E
:10049000941211F00C945602A9EDB1E08C91ACE9E4
:1004A000B1E08D9388278C930C945E02A9EDB1E0A6
:1004B0008C918F5F8C9310F40C94320281E08093C6
:1004C000DA01A4E9B1E088278C93A4E5B1E0E7EA7A
:1004D000F1E0222791E00E94D10FA3EAB1E00C9352
:1004E0000091A301003011F00C947D02A4E5B1E06D
:1004F0000E948C12A3EAB1E08C9381E08093D90131
:100500004091A3010091D901041718F011F00C9447
:10051000D80280E3482FA9EDB1E0AD90BB24A3E55C
:10052000B1E0AA0DBB1D0C91041781E008F480E036
:100530008F9389E3482FA9EDB1E0AD90BB24A3E5EB
:10054000B1E0AA0DBB1D0C91041781E010F009F079
:1005500080E09F918923882311F40C94D002A9EDA7
:10056000B1E0AD90BB24A3E5B1E0AA0DBB1D8C9119
:10057000AAEDB1E0AD90BB24A3E9B1E0AA0DBB1D8B
:100580008C93AAEDB1E08C918F5F8C9380E0AAED03
:10059000B1E0AD90BB24A3E9B1E0AA0DBB1D8C93E3
:1005A000A9EDB1E08C918F5F8C9310F40C948002D4
:1005B000ACE9B1E00D911C910F931F93A4E9B1E058
:1005C0000E944C12402F512F1F910F91040F151FA5
:1005D000ACE9B1E00D931C93A4E5B1E0E7EAF1E0EA
:1005E000222791E00E94D10F002F003018F011F067
:1005F0000C94FC020C9403038091A2018F778093EA
:10060000A2010C9408038091A20180688093A2014A
:10061000A4E5B1E00E948C12082F0F93A4E5B1E08D
:10062000E7EAF1E0222791E00E94D10F402F0F91DD
:10063000041BA3EAB1E00C93A4E5B1E00E948C1284
:10064000EA2FFB2F0091A3013197E01BF0400FEF41
:10065000A4E5B1E00E948412A4E5B1E00E949510E7
:10066000EDE0F0E0AEE9B1E00E947E12ACE9B1E06D
:100670000D911C91013050E0150711F00C945E03B0
:10068000A4E1B1E0ECE8F5E20E94BD0FA4E1B1E025
:100690000E94900EE0E6F0E00E94F611A4E1B1E0C5
:1006A0000E94900EE4E9F5E20E94BD0FA4E1B1E0E2
:1006B0000E94D80E0E94E50E0C94EA03023050E02E
:1006C000150711F00C948203A4E1B1E0E6E9F5E22C
:1006D0000E94BD0FA4E1B1E00E94900EE4E6F0E0BC
:1006E0000E94F611A4E1B1E00E94900EE4E9F5E267
:1006F0000E94BD0FA4E1B1E00E94D80E0E94E50E59
:100700000C94EA03033050E0150711F00C949603A3
:10071000A4E1B1E0EEE9F5E20E94BD0FA4E1B1E091
:100720000E94D80E0E94E50E0C94EA03043050E0BB
:10073000150711F00C94AF0381E08093A4018BE1C5
:100740000E94E80EEAEBF5E20E94DE0E8BE10E94C9
:10075000E80EE0ECF5E20E94DE0E0C94EA030530B0
:1007600050E0150711F00C94BA0380E08093A401C7
:100770000C94EA03063050E0150711F00C94DE03E8
:10078000A4E1B1E0E4ECF5E20E94BD0FA4E1B1E028
:100790000E94900EE8E6F0E00E94FB11A4E1B1E0B7
:1007A0000E94900EE4E9F5E20E94BD0FA4E1B1E0E1
:1007B0000E94D80E0E94E50E0C94EA03A4E1B1E079
:1007C000ECECF5E20E94BD0FA4E1B1E00E94D80E6E
:1007D0000E94E50E089500919901013011F00C94EA
:1007E0001F0480E080939901A4E1B1E03FE30E94FF
:1007F000990EA4E1B1E08C91082F0A3011F00C940D
:100800001D04A4E1B1E00E948C12082F41E0041BFA
:10081000AAE9B1E00C93A4E1B1E00E948C12EA2FA6
:10082000FB2F00919A013197E01BF0400FEFA4E1FC
:10083000B1E00E9484120C94F9030E94C900009157
:10084000A401013011F00C94D7048BE10E94E80E52
:10085000EAEBF5E20E94DE0E8BE10E94E80EE0EC8E
:10086000F5E20E94DE0EE4EEF5E20E94DE0E0E944A
:10087000E50EEAEFF5E20E94DE0E0E94E50EE2E1EF
:10088000F6E20E94DE0EA4E3B7E0E8E8F0E00E94A2
:10089000F6110E94D60E0E94E50EECE1F6E20E94EF
:1008A000DE0EA4E3B7E0ECE9F0E00E94F6110E944E
:1008B000D60E0E94E50EE6E2F6E20E94DE0EA4E30A
:1008C000B7E0E9EAF0E00E94FB110E94D60E0E9418
:1008D000E50EE2E3F6E20E94DE0EA4E3B7E0EAE60C
:1008E000F0E00E94FB110E94D60E0E94E50EE2E4A9
:1008F000F6E20E94DE0EA4E3B7E0E8E6F0E00E9434
:10090000FB110E94D60E0E94E50EEEE4F6E20E9474
:10091000DE0EA4E3B7E0ECE8F0E00E94FB110E94D9
:10092000D60E0E94E50EEEE5F6E20E94DE0EA4E38E
:10093000B7E0EEE8F0E00E94FB110E94D60E0E94A4
:10094000E50EEEE6F6E20E94DE0EA4E3B7E0E5EA8D
:10095000F0E00E94F6110E94D60E0E94E50EE8E734
:10096000F6E20E94DE0EA4E3B7E0E9EBF0E00E94BD
:1009700002120E94D60E0E94E50EE2E8F6E20E9404
:10098000DE0EA4E3B7E0E4EAF0E00E9402120E9467
:10099000D60E0E94E50EECE8F6E20E94DE0E0E9402
:1009A000E50E88EC90E00E94810F0C94B30584E181
:1009B00090E00E94810FE0E9F6E20E94DE0EA4E3DF
:1009C000B7E0E8E8F0E00E94F6110E94D60E0E941F
:1009D000E50E84E190E00E94810FE6E9F6E20E94D4
:1009E000DE0EA4E3B7E0ECE9F0E00E94F6110E940D
:1009F000D60E0E94E50E84E190E00E94810FECE9A2
:100A0000F6E20E94DE0EA4E3B7E0E9EAF0E00E941D
:100A1000FB110E94D60E0E94E50E84E190E00E9438
:100A2000810FE2EAF6E20E94DE0EA4E3B7E0EAE616
:100A3000F0E00E94FB110E94D60E0E94E50E84E1B8
:100A400090E00E94810FE8EAF6E20E94DE0EA4E345
:100A5000B7E0E8E6F0E00E94FB110E94D60E0E948B
:100A6000E50E84E190E00E94810FEEEAF6E20E943A
:100A7000DE0EA4E3B7E0ECE8F0E00E94FB110E9478
:100A8000D60E0E94E50E84E190E00E94810FE4EB17
:100A9000F6E20E94DE0EA4E3B7E0EEE8F0E00E948A
:100AA000FB110E94D60E0E94E50E84E190E00E94A8
:100AB000810FA5EAB0E04D915D916D917C91AAEB1B
:100AC000B0E00D911D912D913C910E94E0110CF42C
:100AD00002C00C947705A5EAB0E00D911D912D910F
:100AE0003C91AAEBB0E00D931D932D933C93EAEB60
:100AF000F6E20E94DE0EA4E3B7E0EAEBF0E00E942B
:100B0000F6110E94D60E0E94E50E84E190E00E944C
:100B1000810FE0ECF6E20E94DE0EA4E3B7E0E9EB21
:100B2000F0E00E9402120E94D60E0E94E50E84E1BF
:100B300090E00E94810FE6ECF6E20E94DE0EA4E354
:100B4000B7E0E4EAF0E00E9402120E94D60E0E9492
:100B5000E50E84E190E00E94810FECE8F6E20E944D
:100B6000DE0E0E94E50E08958FEF8ABD80E088BDFD
:100B700008E114EE23E030E0A4E7B0E00D931D930C
:100B80002D933C9380E08093A400C29A86E990E084
:100B90000E94810FC39A86E990E00E94810FC49A57
:100BA0008AEF90E00E94810FC298C398C49880E0B9
:100BB00090E0AAE6B0E08D939C9301E010E020E085
:100BC00030E0A0E8B0E00D931D932D933C934AE0F4
:100BD00050E060E070E0A0E8B0E00D911D912D9133
:100BE0003C910E94E0111CF011F00C941706AAE64B
:100BF000B0E00D911C910F931F9307B1007E076029
:100C000007B90E94C30F482F592F1F910F91040F4E
:100C1000151FAAE6B0E00D931C9381E090E00E94BE
:100C2000810FA0E8B0E00E942D0E0C94E705AAE623
:100C3000B0E00D911C914AE050E00E94500EAAE6EF
:100C4000B0E04D935C9382E090E00E94810FAAE6B1
:100C5000B0E00D911C91043650E015070CF402C071
:100C60000C94370684E08093B9000C94F50D0E9433
:100C7000840C789489B7816089BF0E94EB030C943F
:100C80003D060F921F922F923F924F925F927F925A
:100C9000AF92BF920F931F932F933F934F935F9306
:100CA0006F937F938F939F93AF93BF93CF93DF9374
:100CB000EF93FF938FB78F93A89584E680935200AC
:100CC0000E9488060E94E7070E94A4080E94D70994
:100CD0000E94810B0E94090C8F918FBFFF91EF91B1
:100CE000DF91CF91BF91AF919F918F917F916F9144
:100CF0005F914F913F912F911F910F91BF90AF90B6
:100D00007F905F904F903F902F901F900F9018957D
:100D100007B1007E056007B90E94C30FA4E6B0E0EA
:100D20008D939D9388278D938C9300E014E020E0B1
:100D300030E0A4E6B0E04D915D916D917C910E9410
:100D4000DB11A4E6B0E00D931D932D933D9307B105
:100D5000007E036007B90E94C30FA0E6B0E08D9348
:100D60009D9388278D938C9307B1007E006007B90F
:100D70000E94C30FA8E6B0E08D939C9307B1007E5C
:100D8000066007B90E94C30FA9EAB0E08D939C9357
:100D900000E014E00F931F9307B1007E076007B9CE
:100DA0000E94C30F482F592F1F910F91041B150B41
:100DB000AAE6B0E00D931C93ACE6B0E00D911D9156
:100DC0002D913C914AEF50E060E070E00E94190FD5
:100DD000A0E8B0E04D935D936D937D93ACE6B0E0F9
:100DE0000D911D912D913C91A0E8B0E04D915D9148
:100DF0006D917C910E94DB11ACE6B0E00D931D93E8
:100E00002D933D93A0E6B0E00D911D912D913C9165
:100E1000A5EBB0E04D915C91662777270E94DB112E
:100E2000A0E8B0E00D931D932D933D93ACE6B0E0A8
:100E30000D911D912D913C91A0E8B0E04D915D91F7
:100E40006D917C910E94D611ACE6B0E00D931D939C
:100E50002D933D93A0E7B0E00D911D912D913C9114
:100E60004AEF50E060E070E00E94190FACE7B0E09C
:100E70004D935D936D937D93A0E7B0E00D911D912F
:100E80002D913C91ACE7B0E04D915D916D917C91DD
:100E90000E94DB11A0E7B0E00D931D932D933D93CD
:100EA000A0E7B0E00D911D912D913C91A4E6B0E03A
:100EB0004D915D916D917C910E94D611A0E7B0E0BB
:100EC0000D931D932D933D93A0E7B0E00D911D91DF
:100ED0002D913C9149E150E060E070E00E94190FD3
:100EE000ACE7B0E04D935D936D937D93A4E6B0E0E5
:100EF0000D911D912D913C914AE050E060E070E031
:100F00000E949A0FA0E8B0E00D931D932D933D939E
:100F1000ACE7B0E00D911D912D913C91A0E8B0E0BF
:100F20004D915D916D917C910E94DB11ACE7B0E039
:100F30000D931D932D933D93ACE7B0E00D911D9162
:100F40002D913C9143E250E060E070E00E949A0FE6
:100F5000ACE7B0E00D931D932D933D93ACE7B0E06B
:100F60000D911D912D913C9144E650E060E070E0C0
:100F70000E94190FACE9B0E04D935D936D937D93A2
:100F8000ACE6B0E00D911D912D913C91ACE9B0E043
:100F90004D915D916D917C910E94D611ACE6B0E0CF
:100FA0000D931D932D933D93ACE6B0E00D911D91F3
:100FB0002D913C9149E150E060E070E00E94190FF2
:100FC000A8E8B0E04D935D936D937D930895A8E8F4
:100FD000B0E00D911D912D913C91A8E9B0E04D91AB
:100FE0005D916D917C910E94D611A0EAB0E00D93C5
:100FF0001D932D933D93ACE9B0E00D911D912D9182
:101000003C91A0EAB0E04D915D916D917C910E9480
:10101000D611A0EAB0E00D931D932D933D93A0EA65
:10102000B0E00D911D912D913C9141E150E060E0C7
:1010300070E00E949A0FA0EAB0E00D931D932D93EB
:101040003D93A5EAB0E00D911D912D913C91A0EA50
:10105000B0E04D915D916D917C910E94D611A5EA11
:10106000B0E00D931D932D933D9348ED56ED60E058
:1010700070E0A5EAB0E00D911D912D913C910E9488
:10108000E0111CF011F00C9447080C94510808ED85
:1010900016ED20E030E0A5EAB0E00D931D932D930E
:1010A0003C9348E259E26FEF7FEFA5EAB0E00D9183
:1010B0001D912D913C910E94E0110CF402C00C9402
:1010C0006B0808E219E22FEF3FEFA5EAB0E00D93BD
:1010D0001D932D933C93A5EAB0E00D911D912D91A8
:1010E0003C914BE950E060E070E00E94190FA0E8ED
:1010F000B0E04D935D936D937D93A0EAB0E00D91C8
:101100001D912D913C9145EA50E060E070E00E9415
:10111000190FACE7B0E04D935D936D937D93A0E81C
:10112000B0E00D911D912D913C91ACE7B0E04D9157
:101130005D916D917C910E94D611A0E9B0E00D9374
:101140001D932D933D930895A3EBB0E00D911D9158
:1011500017FB1EF42FEF3FEF02C022273327A9EA27
:10116000B0E04D915D9157FB1EF46FEF7FEF02C031
:10117000662777270E94DB11AFEAB0E00D931D933D
:101180002D933D93A5EAB0E00D911D912D913C91D9
:1011900040E25EE460E070E00E94190FACE7B0E06E
:1011A0004D935D936D937D93ACE7B0E00D911D91F0
:1011B0002D913C910E946D0FACE7B0E00D931D9313
:1011C0002D933D9341E050E060E070E0ACE7B0E08B
:1011D0000D911D912D913C910E94E0110CF402C0E3
:1011E0000C94FC0801E010E020E030E0ACE7B0E057
:1011F0000D931D932D933C93AFEAB0E00D911D919B
:101200002D913C91ACE7B0E04D915D916D917C9159
:101210000E94190FAFEAB0E04D935D936D937D93FB
:10122000A5EAB0E00D911D912D913C9140ED57E064
:1012300060E070E00E94190FACE7B0E04D935D9361
:101240006D937D93ACE7B0E00D911D912D913C9194
:101250000E946D0FACE7B0E00D931D932D933D936D
:1012600046E150E060E070E0ACE7B0E00D911D9128
:101270002D913C910E94E0111CF011F00C94420958
:101280000C944C0906E110E020E030E0ACE7B0E05F
:101290000D931D932D933C930BE110E020E030E083
:1012A000ACE7B0E04D915D916D917C910E94DB11B6
:1012B000ACE7B0E00D931D932D933D93ACE7B0E008
:1012C0000D911D912D913C914FEF5FEF6FEF7FEFEF
:1012D0000E949A0FA4E8B0E00D931D932D933D93C7
:1012E000ACE7B0E04D915D916D917C91AFEAB0E0DB
:1012F0000D911D912D913C910E94E0111CF011F077
:101300000C9484090C949009ACE7B0E00D911D9108
:101310002D913C91AFEAB0E00D931D932D933C933A
:10132000A4E8B0E04D915D916D917C91AFEAB0E0A1
:101330000D911D912D913C910E94E0110CF402C081
:101340000C94AE09A4E8B0E00D911D912D913C9153
:10135000AFEAB0E00D931D932D933C93AFEAB0E05C
:101360000D911D912D913C91A4E9B0E00D931D9339
:101370002D933C93A0E9B0E00D911C91A4E9B0E05D
:101380004D915C91041B150BACE8B0E00D931C93E0
:10139000A0E9B0E00D911C91A4E9B0E04D915C9101
:1013A000040F151FAEE8B0E00D931C930895009153
:1013B000A400003011F00C94430A80E090E0ACE807
:1013C000B0E08D939C9380E090E0AEE8B0E08D9328
:1013D0009C9300E010E020E030E0A0E9B0E00D9345
:1013E0001D932D933C9300E010E020E030E0A8E94D
:1013F000B0E00D931D932D933C9300E010E020E0AE
:1014000030E0A5EAB0E00D931D932D933C9300E0EE
:1014100010E020E030E0ACE6B0E00D931D932D939A
:101420003C9300E010E020E030E0A8E8B0E00D934D
:101430001D932D933C9300E010E020E030E0ABEAF8
:10144000B0E00D931D932D933C93AAE6B0E00D916F
:101450001C91023350E015071CF011F00C94320A75
:101460000C94410A0E94840C81E08093A40000E067
:1014700010E020E030E0ABEAB0E00D931D932D9337
:101480003C930C94800B013011F00C94570AAAE69F
:10149000B0E00D911C91023350E015070CF402C02E
:1014A0000C94550A83E08093A4000C94800B0330C5
:1014B00011F00C947D0BABEAB0E00E942D0E43E0DE
:1014C00050E060E070E0A0E9B0E00D911D912D9139
:1014D0003C910E94E01180E014F009F081E08F93CC
:1014E00044E650E060E070E0ABEAB0E00D911D91A1
:1014F0002D913C910E94E01180E00CF481E09F91DD
:101500008923882311F40C94AB0AA0E9B0E04D9133
:101510005D916D917C91A8E9B0E00D911D912D91A7
:101520003C910E94E0110CF402C00C94A90AA8E9B5
:10153000B0E00D911D912D913C9142E050E060E0B2
:1015400070E00E94D611A8E9B0E00D931D932D9391
:101550003D930C947B0B4DEF5FEF6FEF7FEFA0E9B6
:10156000B0E00D911D912D913C910E94E0110CF481
:1015700002C00C94E30AA0E9B0E04D915D916D9139
:101580007C91A8E9B0E00D911D912D913C910E94B4
:10159000E0111CF011F00C94CF0A0C94E10AA8E9B8
:1015A000B0E00D911D912D913C9142E050E060E042
:1015B00070E00E94DB11A8E9B0E00D931D932D931C
:1015C0003D930C947B0B81B5886181BD877F81BD84
:1015D00000E010E020E030E0ABEAB0E00D931D93B6
:1015E0002D933C9301E010E020E030E0ACE7B0E068
:1015F0000D931D932D933C934FEF50E060E070E00E
:10160000ACE7B0E00D911D912D913C910E94E0114D
:101610001CF011F00C94750BACE8B0E00D911C912E
:10162000003050E0150781E009F080E08F93AEE8CC
:10163000B0E00D911C91003050E0150781E009F0F9
:1016400080E09F918923882311F40C94290B0C943A
:10165000750BACE8B0E00D911C91003050E015071F
:101660001CF011F00C94360B0C943A0BACE8B0E083
:101670000E94430EACE8B0E00D911C91003050E0A8
:1016800015070CF402C00C94490BACE8B0E00E94C2
:101690003C0EAEE8B0E00D911C91003050E0150713
:1016A0001CF011F00C94560B0C945A0BAEE8B0E001
:1016B0000E94430EAEE8B0E00D911C91003050E066
:1016C00015070CF402C00C94690BAEE8B0E00E9460
:1016D0003C0E89E190E00E94810F0E94810BACE7F3
:1016E000B0E00E942D0E0C94FC0A80E08093A400D0
:1016F00081B5886081BD0C94800B83E08093A40049
:101700000895ACE8B0E00D911C91043B50E0150742
:101710001CF011F00C948E0B0C94960B84EB90E063
:10172000ACE8B0E08D939C930C94A70BACE8B0E0D0
:101730000D911C910C345FEF15070CF402C00C9452
:10174000A70B8CE49FEFACE8B0E08D939C93AEE8E0
:10175000B0E00D911C91043B50E015071CF011F016
:101760000C94B40B0C94BC0B84EB90E0AEE8B0E0AE
:101770008D939C930C94CD0BAEE8B0E00D911C9131
:101780000C345FEF15070CF402C00C94CD0B8CE405
:101790009FEFAEE8B0E08D939C93ACE8B0E00D9184
:1017A0001C91003050E015070CF402C00C94DB0BC8
:1017B000969A0C94DC0B9698AEE8B0E00D911C91D3
:1017C000003050E015070CF402C00C94EA0B979A15
:1017D0000C94EB0B9798ACE8B0E08D919C910E9433
:1017E000700EA8E7B0E08D939C93AEE8B0E08D91C9
:1017F0009C910E94700EAAE7B0E08D939C930FEF2E
:1018000040917800041B0ABDAAE7B0E08C9188BD26
:101810000895A4E7B0E00D911D912D913C914AEF00
:1018200050E060E070E00E94190FACE7B0E04D932B
:101830005D936D937D93A4E7B0E00D911D912D9183
:101840003C91ACE7B0E04D915D916D917C910E942F
:10185000DB11A4E7B0E00D931D932D933D93A4E716
:10186000B0E00D911D912D913C91A8E6B0E04D9115
:101870005D9157FB1EF46FEF7FEF02C0662777275D
:101880000E94D611A4E7B0E00D931D932D933D93D4
:1018900048E154EE63E070E0A4E7B0E00D911D91E3
:1018A0002D913C910E94E0111CF011F00C945A0C07
:1018B0000C945D0CC29AC398C49848E154EE63E05E
:1018C00070E0A4E7B0E00D911D912D913C910E9434
:1018D000E0110CF402C00C94700CC39AC498C29826
:1018E00040E859EA63E070E0A4E7B0E00D911D9193
:1018F0002D913C910E94E0110CF402C00C94830CD9
:10190000C398C298C49A089581B5886181BD877FC4
:1019100081BD80E090E0A9EAB0E08D939C9301E066
:1019200010E020E030E0A0E8B0E00D931D932D938F
:101930003C934AE050E060E070E0A0E8B0E00D9138
:101940001D912D913C910E94E0111CF011F00C941E
:10195000C90CA9EAB0E00D911C910F931F9307B138
:10196000007E066007B90E94C30F482F592F1F91B0
:101970000F91040F151FA9EAB0E00D931C9381E0AD
:1019800090E00E94810FA0E8B0E00E942D0E0C9420
:10199000990CA9EAB0E00D911C914AE050E00E9438
:1019A000500EA3EBB0E04D935C9300E010E020E01C
:1019B00030E0A4E6B0E00D931D932D933C9301E03D
:1019C00010E020E030E0A0E8B0E00D931D932D93EF
:1019D0003C9344E650E060E070E0A0E8B0E00D9198
:1019E0001D912D913C910E94E0111CF011F00C947E
:1019F000360D07B1007E056007B90E94C30FACE742
:101A0000B0E08D939D9388278D938C9300E014E034
:101A100020E030E0ACE7B0E04D915D916D917C91BC
:101A20000E94DB11ACE7B0E00D931D932D933D9325
:101A3000A4E6B0E00D911D912D913C91ACE7B0E092
:101A40004D915D916D917C910E94D611A4E6B0E01C
:101A50000D931D932D933D9382E090E00E94810FA2
:101A6000A0E8B0E00E942D0E0C94E90CA4E6B0E0D2
:101A70000D911C9144E650E00E94760EA7EBB0E079
:101A80004D935C930AEF10E020E030E0A7EBB0E06C
:101A90004D915C91662777270E949A0FA0E7B0E0EE
:101AA0000D931D932D933D9300E010E020E030E076
:101AB000A0E6B0E00D931D932D933C9301E010E060
:101AC00020E030E0A0E8B0E00D931D932D933C930F
:101AD00044E650E060E070E0A0E8B0E00D911D91B8
:101AE0002D913C910E94E0111CF011F00C94A30D7B
:101AF00007B1007E036007B90E94C30FACE7B0E0F6
:101B00008D939D9388278D938C93A0E6B0E00D91E3
:101B10001D912D913C91ACE7B0E04D915D916D919F
:101B20007C910E94D611A0E6B0E00D931D932D93F9
:101B30003D9382E090E00E94810FA0E8B0E00E9417
:101B40002D0E0C94680DA0E6B0E00D911C9144E6BA
:101B500050E00E94760EA5EBB0E04D935C9381B50A
:101B6000886081BDA5EBB0E00D911C91003951E07A
:101B7000150710F00C94C10D83E08093B9000C940C
:101B8000F50DA5EBB0E00D911C91083552E015075D
:101B900018F011F00C94CE0D0C94D30D83E08093CB
:101BA000B9000C94F50DA7EBB0E00D911C910E352A
:101BB00051E0150710F00C94E20D82E08093B9001B
:101BC0000C94F50DA7EBB0E00D911C910E3E52E088
:101BD000150718F011F00C94EF0D0C94F40D82E041
:101BE0008093B9000C94F50D089581B5886181BD8D
:101BF000877F81BD01E010E020E030E0A0E8B0E0A8
:101C00000D931D932D933C93A9EBB0E04C91552778
:101C100066277727A0E8B0E00D911D912D913C91AA
:101C20000E94E0111CF011F00C94260EC49A86E973
:101C300090E00E94810FC49886E990E00E94810F95
:101C4000A0E8B0E00E942D0E0C94040EE2E0F0E05B
:101C50000E94100F0C94FA0D08950D911D912D9175
:101C60003C9181E0080F8827181F281F381F3C93DC
:101C70002E931E930E930895ED91FC91EF5FFF4F0D
:101C8000FC93EE930895ED91FC91E150F040FC93AC
:101C9000EE93089509D00E94900F00FC10D0089593
:101CA00003D024D001F8F9CF0024E89457FF02C0F4
:101CB00009D0689400F80BD010F80124089502D0E0
:101CC00009D00895509540954F5F5F4F0895E8946F
:101CD00017FF0895009510950F5F1F4F68940895A2
:101CE00099231AF48095909501960895352F242F05
:101CF000E894452B11F468940895512F402F002744
:101D0000112780E1440F551F001F111F021B130BE9
:101D1000416018F4020F131F4E7F8A9599F70895BA
:101D20008F938D918823E9F711978F910895A4E3FC
:101D3000B7E018D0883091F08D3039F03323C9F3F3
:101D40008D933A9563FE44D0F4CF63FC04C08DE0DC
:101D50003FD08AE03DD088278C93089539D01197E1
:101D60003395E7CF0F929F93AF93BF937F9380916B
:101D7000E8008823E1F3F8948091E8008A95809345
:101D8000E8009091E600AEEBB0E0A90F0024B01D92
:101D90008C919395983209F499279093E600789462
:101DA0007F91BF91AF919F910F900895A4E3B7E009
:101DB0008D91882311F00CD0FBCF08950E949110D3
:101DC000802D11F005D0FACF08958DE001D08AE082
:101DD0009F939FB79F93AF93BF930F937F939091E0
:101DE00013019832E1F3F894909113019395909335
:101DF0001301992700911201A9EEB0E0A00FB91FBD
:101E00008C930395083209F4002700931201559A28
:101E10007F910F91BF91AF919F919FBF9F91089527
:101E200088EE93E06ED03197D9F7089500FC05D085
:101E3000089530D005D001F8F9CF37D03FD00895BC
:101E4000842F952FA62FB72FE894452B462B472B91
:101E500011F468940895402F512F622F732F00279B
:101E6000112722273327F0E2440F551F661F771FE3
:101E7000001F111F221F331F081B190B2A0B3B0BBE
:101E8000416028F4080F191F2A1F3B1F4E7FFA9547
:101E900059F708950024E89477FF02C006D06894AB
:101EA00000F809D010F80124089512D04F5F5F4F59
:101EB0006F4F7F4F0895E89437FF08950095109570
:101EC000209530950F5F1F4F2F4F3F4F6894089517
:101ED0004095509560957095089537FF0895009549
:101EE0001095209530950F5F1F4F2F4F3F4F08954E
:101EF0003197F1F70895689462F80895E89462F8CC
:101F00000895EF93FF93EE27E82BE92B31F0E0EAF9
:101F1000FFE03197F1F70197D1F7FF91EF91089525
:101F20000F92B801469F8001479F100D569F100DDC
:101F30000F9008950F921F922F92C801D901489FC8
:101F400080014A9F90014B9F202C499F100D211D1D
:101F5000321D5A9F202C589F100D211D321D599F54
:101F6000200D311D689F200D311D699F300D789F18
:101F7000300D2F901F900F9008950E9491100D9298
:101F80000020D9F70895369A3699FECF369A3699B9
:101F9000FECF84B195B1089599910027A90FB01F84
:101FA0001197492F4A955E2F6F2FE894112743957B
:101FB000203019F0C895802D01C080818823B9F0A8
:101FC0007C917723A1F0781739F40EF0042F139544
:101FD000689411963196EBCF112321F0411BA11B80
:101FE0001127B10BE894E52FF62F1196E0CF882347
:101FF00011F0002708950895D190E190F19001919A
:10200000089521913191419151910895102F90E8B7
:10201000FF0C001F0927990FF7941078652F90E89F
:10202000440F551F5927990F479560780038089538
:10203000FF0C90E89027110F9795F794092F0895BA
:10204000502F2D2D3E2D4F2D612F08952DEC3CEC62
:102050004CEC5DE366270FC0CFDFF2DFDD24EE241A
:1020600090E8F92E0FE307C0CCDF05C02227332705
:1020700040E251E46627552351F1002381F1C6DF88
:1020800071F11627005850580894050B18F407FDF5
:1020900003C025C007FD23C0469537952795F694C4
:1020A000E794D79422D0FF202AF0DD0CEE1CFF1C11
:1020B000015073F09D2D969548F0DD203AF4EE2006
:1020C0002AF491E0D90E9927E91EF91EB1CF07C075
:1020D0009FE7092FF92A9FEFD92EE92E0895DD24D5
:1020E000EE24FF240027112708959F929924AA2403
:1020F000BB2488E1D216E306F40628F0D21AE30ADC
:10210000F40A089401C08894991CAA1CBB1CDD0C1D
:10211000EE1CFF1C8A9571F7D92CEA2CFB2C9F90A2
:102120000895C8953196002008950E947E0FE89486
:1021300088278A938A93D3DF11278D918032E9F320
:102140001197BBD098F08D3229F4109511968C918F
:10215000B4D060F08E3229F411968C91AED008F490
:1021600046C022960E947B0F81E008958C91A5D0F5
:10217000D8F547D01196D0F703958D919ED0E0F316
:102180008E3229F48C9199D010F41196FBCF8534BE
:1021900019F0853609F055C011968C918ED060F0FB
:1021A0008D3219F08B3221F0DCCF08800094088248
:1021B00011968C9182D0A8F68053898311968C91C8
:1021C0007CD058F49981990F990F0980900D990F3F
:1021D0008053890F8983873220F6898198819923DA
:1021E0000AF48195080F2DC08E3289F611968C91D4
:1021F00064D068F606D018F011960A95F8CF1196BB
:10220000C1CF4F2D3E2D2D2DDD0CEE1CFF1CA8F057
:10221000DD0CEE1CFF1C88F0D20EE31EF41E68F0ED
:10222000DD0CEE1CFF1C48F0805309F06894D80EBA
:102230008827E81EF81E08F00895F42EE32ED22E0B
:10224000089534D019F116F5098308E921D00695CF
:10225000882787959F2D9F77980FF92E0150000FA3
:10226000110F07958981882379F01AF48195898364
:1022700006C0ECDE89818A958983D9F705C0F6DE30
:1022800089818A958983D9F72296089528DFFCCF22
:102290000DD041F0FF2032F00A9531F0DD0CEE1C3C
:1022A000FF1CD2F7889408950894089500240D28FF
:1022B0000E280F28002A00200895803320F08A334A
:1022C00010F4089408958894089591E005C092E070
:1022D00003C094E001C098E024DF0D929A95E1F7E5
:1022E0000895819104D08D938823D9F7089581367C
:1022F00018F08B3708F48F7D08957F930F93AF9379
:10230000BF938F939F938FB78F93E8948091E8004A
:1023100008E2081B21F49CB10E947B0F13C00091BE
:10232000E700AEEBB0E077279CB1A00FB71F9C93FE
:10233000689483958093E8000395083209F4002798
:102340000093E7009D3011F40E94C5008F918FBF6C
:102350009F918F91BF91AF910F917F9118957F932E
:10236000AF93BF938F939F938FB78F9390911301E8
:10237000992399F09A95909313019927A9EEB0E0CB
:1023800080911101A80FB91F9C918395883209F49F
:102390008827809311019CB901C055988F918FBFF8
:1023A0009F918F91BF91AF917F911895040F151F49
:1023B000261F371F0895041B150B260B370B089596
:1023C00004171507260737070895000F111F221F4E
:1023D000331F089500951095209530950F5F1F4F7E
:1023E0002F4F3F4F0895019110810EC0019111911F
:1023F000219130810BC00191108117FF05C03FEF83
:102400002FEF04C0008111272227332737FF03C095
:10241000E1DF8DE28D93CF93DF93CF92DF92EF9246
:10242000AA24BB24CC24DD24EE2440E2CAE0DD272C
:1024300055E093E38881890F87FD9F7083FD907F2E
:10244000891B89935A95A9F7C0DFAA1CBB1CCC1C19
:10245000DD1CEE1C4A9551F7E894EFE0FF278291CE
:102460000ED0EB30E0F71EF068948A2D0CD0882750
:102470008D93EF90DF90CF90DF91CF910895982FBB
:10248000829501D0892F8F70805D26F0803309F40A
:10249000089568948D9308950027112722273327E4
:1024A0001DD08A3328F4803318F005D015D0F9CF29
:1024B0000EF490CF089580538F93402F512F622FA9
:1024C000732F83DF82DF72DF80DF8F919927080F00
:1024D000191F291F391F08958D910895E894FCDF75
:1024E0008032E9F38B32D9F38930C9F38D3211F49C
:1024F0006894F2CF089588278D93089594E0819190
:102500008D939A95E1F7089581918D930A9519F02D
:102510008823D1F70895EFCF8FEF83959D9199236D
:10252000E1F70895689401C0E894AF93BF938D914B
:1025300016F0919103C00E949110902D891718F008
:1025400011F48823A1F7BF91AF910895689463F8BF
:102550000895000000003A003D00414458004944FD
:10256000470049444E0054454C00535450005357C3
:102570004900424154004D4F41004D4F42005354D9
:102580005200455252004D4F44002A0023303A4138
:1025900044583D00210023303A4944473D00233050
:1025A0003A49444E3D5B4350552D4D6F64756C2048
:1025B000574F463130325D2100005B313B316600C0
:1025C0005B324A0023303A4241543D0023303A45C1
:1025D00052523D5B53796E746178204572726F720E
:1025E0005D2100002354656C656D657472792076F9
:1025F000312E3020202020202000232020202020C9
:1026000020202020202020202020202020202020CA
:1026100000002354696C74203D2000002347797228
:102620006F203D20000023526F636B6572203D20B8
:10263000000023466F6F74737769746368203D20D0
:1026400000002342617474657279203D2000234D9F
:102650006F746F72206C656674203D200000234DFE
:102660006F746F72207269676874203D2000235375
:10267000747265DF203D2000234572726F72203D29
:102680002000234D6F6465203D200000313A340066
:10269000323A313D0000323A333D0000323A353DA6
:1026A0000000323A363D0000323A373D0000323AFF
:1026B000383D0000323A393D0000323A31303D00B9
:0C26C000323A31313D00323A31323D00F7
:00000001FF
